:100000000C9411060C945F280C948C280C943906DF
:100010000C9439060C9439060C9439060C94390664
:100020000C9439060C9439060C94B60C0C943906D1
:100030000C9439060C9439060C9439060C94390644
:100040000C94B9280C9439060C94512C0C948C2CDB
:100050000C9439060C9439060C9439060C94390624
:100060000C9439060C943906C71BCE1BCE1BC71B3C
:10007000CE1BCE1BCE1BCE1BCE1BCE1BCE1BCE1B38
:10008000CE1BCE1BCE1BCE1BCE1B3C1BCE1BCE1BBA
:10009000CE1BCE1BCE1B9F1ACE1BCE1BCE1BCE1B48
:1000A000CE1BCE1BCE1BCE1BCE1BCE1BCE1BCE1B08
:1000B000CE1BCE1BCE1B481B481B481B481B481B96
:1000C000481B481B481B481BCE1BCE1BCE1BCE1B00
:1000D000CE1BCE1BA41A471B471B471B471BCE1B1F
:1000E000581B601B681B701B781B801B881B901B98
:1000F0009A1BA41BAE1BB81BEB1AAB1ACE1BCE1B54
:10010000CE1BCE1B3C1BCE1BCE1BCE1BCE1BCE1B39
:10011000CE1BCE1BCE1B461B461B461B461BCE1BB7
:10012000581B601B681B701B781B801B881B901B57
:100130009A1BA41BAE1BB81BEB1AAB1ACE1BCE1B13
:10014000CE1BCE1B3C1BFF1BFF1BFF1BFF1BFF1B04
:10015000FF1BFF1BFF1BFF1BFF1BFF1BFF1BFF1BCF
:10016000201D201D201D201D201D201D461C501C53
:100170005A1C641CCA1CD41CE21CF41C911D011ED8
:10018000D21DD71DDC1DE11DE61DEB1DF01D011E5E
:10019000FB1DDF24F4240025092516253C254425D4
:1001A00067255425456E746572206D656E752E2E1B
:1001B0002E00546F67676C6564206D6963726F50C1
:1001C000504D00546F67676C656420696E76657288
:1001D0007465642050504D2100546F67676C6564EE
:1001E000205458206D7574696E672100546F6767DD
:1001F0006C65642074656C656D657472792100505E
:10020000726F746F636F6C206572726F72207769A2
:1002100074682052580054696D656F757420776852
:10022000656E20636F6E6E656374696E6720746FB0
:1002300020525800507265737320616E79206B658F
:100240007920746F2063616E63656C00436F6E6E1E
:10025000656374696E6720746F2052582C20706F2C
:100260007765722075702074686520525820287751
:100270006974682062696E6420706C7567206966B5
:10028000206E6F74207573696E6720616C77617979
:10029000732062696E642900546F67676C6564201F
:1002A00027696D6D656469617465206F757470751B
:1002B000742700546F67676C65642027736C6176E0
:1002C00065206D6F64652700546F67676C656420F7
:1002D00027616C776179732062696E642700546FBF
:1002E00067676C65642050504D206368616E6E6571
:1002F0006C206C696D6974005365742052535349C6
:1003000020696E6A656374696F6E206368616E6EE2
:10031000656C2028303D3D64697361626C6529001D
:100320005365742050504D206D696E696D756D2058
:1003300073796E630053657420626561636F6E202C
:10034000696E74657276616C0053657420626561D4
:10035000636F6E2064656C6179005365742062651B
:1003600061636F6E206672657175656E6379206971
:100370006E20487A3A20303D64697361626C652C66
:100380002050783D504D52206368616E6E656C2040
:10039000782C2046783D465253206368616E6E6526
:1003A0006C2078005365742050574D2073746F7023
:1003B0002064656C61792028302064697361626C07
:1003C00065642C20312D323535203D3D20302E31D5
:1003D00073202D2035306D696E29005365742050CF
:1003E000504D2073746F702064656C6179202830E3
:1003F0002064697361626C65642C20312D3235355F
:10040000203D3D20302E3173202D2035306D696E1A
:100410002900536574206661696C736166652064A8
:10042000656C61792028302064697361626C656451
:100430002C20312D323535203D3D20302E3173209A
:100440002D2035306D696E29002A2A2A2A2A2A2A67
:100450002A2A2A2A2A2A2A2A2A2A2A2A2A2A2A2AFC
:100460002A2A2A2A2A2A0052582041636B656420CE
:100470002D2072657665727420737563636573737E
:1004800066756C21002A2A2A2A2A2A2A2A2A2A2A36
:100490002A2A2A2A2A2A2A2A2A2A2A2A2A2A2A2ABC
:1004A0002A2A002A2A2A2A2A2A2A2A2A2A2A2A2AD6
:1004B0002A2A2A2A2A2A2A2A2A2A2A2A2A2A2A2A9C
:1004C0000052582041636B6564202D207570646173
:1004D0007465207375636365737366756C21002A98
:1004E0002A2A2A2A2A2A2A2A2A2A2A2A2A2A2A2A6C
:1004F0002A2A2A2A2A2A2A2A2A2A2A2A0056616CE1
:1005000069642063686F69636573206172653A206E
:100510005B315D2D5B31365D20286368616E6E65F1
:100520006C20312D31362900536574206F7574703D
:10053000757420666F7220706F727420005B585D56
:100540002061626F7274206368616E6765732061F9
:100550006E64206578697420525820636F6E6669F6
:1005600067005B535D207361766520736574746901
:100570006E677320746F205258005B525D20726565
:10058000766572742052582073657474696E67734F
:1005900020746F2064656661756C747300557365B3
:1005A000206E756D62657273205B312D445D207421
:1005B0006F206564697420706F727473205B452DC1
:1005C000515D20666F722073657474696E67730085
:1005D000202D20726563656976657220636F6E6693
:1005E0006967757261746F722C207278207377203E
:1005F000000A0A6F70656E4C52536E672000536597
:10060000742073657269616C2062617564726174D3
:10061000653A200056616C69642063686F696365A0
:10062000733A2031202D20342B34202F2032202DDE
:100630002038202F2033202D20382B34202F203419
:10064000202D203132202F2035202D2031322B3407
:10065000202F2036202D203136005365742043682A
:10066000616E6E656C20636F6E6669673A20005339
:1006700065742044617461726174652028302D3284
:10068000293A200053657420486F70206368616EBA
:100690006E656C7320286D61782032342C20736570
:1006A0007061726174656420627920636F6D6D6141
:1006B00073292076616C69642076616C756573209E
:1006C000312D3235353A2000536574206368616EF0
:1006D0006E656C2073706163696E672028783130B5
:1006E0006B487A293A200053657420524620706F77
:1006F0007765722028302D37293A20005365742001
:100700005246206D616769632028686578292065F5
:100710002E672E20307844454144463030443A20FC
:10072000005365742062617365206672657175653A
:100730006E63792028696E20487A293A20005B5A36
:100740005D20656E74657220726563656976657299
:1007500020636F6E66696775726174696F6E20756C
:1007600074696C79005B465D20646973706C6179B3
:100770002061637475616C206672657175656E6366
:100780006965732075736564005B525D2063616CFD
:1007900063756C6174652072616E646F6D206B654A
:1007A0007920616E6420686F70206C697374005BDF
:1007B000495D207265696E697469616C697A65204A
:1007C00073657474696E677320746F20736B6574DE
:1007D00063682064656661756C7473005B585D20A6
:1007E000726576657274206368616E6765732061F7
:1007F0006E642065786974206D656E75005B535D6D
:1008000020736176652073657474696E67732074F4
:100810006F20454550524F4D20616E6420657869C8
:1008200074206D656E7500557365206E756D62651B
:100830007273205B302D395D20746F20656469749C
:1008400020706172616D657465727300202D205394
:10085000797374656D20636F6E6669677572617414
:10086000696F6E000A0A6F70656E4C52536E672096
:10087000005129204F7574707574206265666F721F
:1008800065206C696E6B20283D465329203A200074
:10089000502920536C617665206D6F646520286552
:1008A00078706572696D656E74616C293A20004FCD
:1008B000292054696D65642042494E4420617420AA
:1008C0007374617274757020203A20004E29205094
:1008D000504D206F7574707574206C696D69746506
:1008E0006420202020203A200044495341424C45B6
:1008F00044004D292050504D205253534920746FCD
:10090000206368616E6E656C202020203A20004CC8
:10091000292050504D206D696E696D756D20737979
:100920006E63202875732920203A200044495341E2
:10093000424C4544004B29204661696C73616665F1
:1009400020626561636F6E20696E74762E20283197
:100950002D32353573293A20004A29204661696CC9
:100960007361666520626561636F6E2064656C61AA
:10097000792028302D323535203D3E20313073200E
:100980002D203135306D696E293A200049292046E5
:1009900061696C7361666520626561636F6E206674
:1009A00072712E203A200048292050574D20737430
:1009B0006F702064656C6179202020202020203A0F
:1009C000200047292050504D2073746F70206465BB
:1009D0006C6179202020202020203A200046292008
:1009E0004661696C736166652064656C617920207D
:1009F00020202020203A200050574D206368616E4F
:100A00006E656C200066756E6374696F6E3A2000C7
:100A10002920706F727420004454462055484620A7
:100A200033322D6269742031306368004F70656E17
:100A30004C52536E675258206D696E6920342F36C0
:100A4000636800466C7974726F6E2F4F72616E67C7
:100A50006552582055484620386368005258207423
:100A60007970653A200044697361626C656400487E
:100A70007A00203D3D200043616C63756C617465B4
:100A800064207061636B657420696E746572766151
:100A90006C3A20004229204D6963726F20286861FA
:100AA0006C66292050504D202020203A00412920FA
:100AB000496E7665727465642050504D20696E20D1
:100AC000202020203A003029204D75746520627561
:100AD0007A7A657220286D6F73746C79293A0039BF
:100AE000292053657269616C20626175647261745A
:100AF000653A00736D617274506F72740046725380
:100B00006B79005472616E73706172656E7400442B
:100B1000697361626C65640038292054656C656D89
:100B2000657472793A202020202020200037292067
:100B30004368616E6E656C20636F6E6669673A200C
:100B40002000362920446174617261746520283068
:100B50002D32293A20202000352920486F7020634B
:100B600068616E6E656C733A202020202000342965
:100B7000204368616E6E656C2073706163696E6797
:100B80003A202000332920524620706F776572206A
:100B900028302D37293A20202000322920524620A3
:100BA0006D616769633A20202020202020202000EA
:100BB00031292042617365206672657175656E63C7
:100BC000793A2020200000000000240027002A009D
:100BD00000000000250028002B000000000023007A
:100BE000260029000404040404040404020202028E
:100BF00002020303030303030102040810204080E0
:100C0000010204081020010204081020000000075F
:100C100000020100000304060000000000000000C4
:100C2000342E11241FBECFEFD8E0DEBFCDBF13E0BE
:100C3000A0E0B1E0EAEAFEE502C005900D92A63917
:100C4000B107D9F716E0A6E9B3E001C01D92A934B7
:100C5000B107E1F71CE0C2E2DCE004C02297FE012C
:100C60000E94302FC032D107C9F70E94792E0C9410
:100C7000532F0C940000A0E0B0E0E1E4F6E00C9407
:100C8000FF2EEC01A880B980CA80DB80A114B104DA
:100C9000C104D10441F484E2A82E89EDB82E8BE57D
:100CA000C82E87E0D82EC601B5012DE133EF41E013
:100CB00050E00E94DC2E27EA31E440E050E00E9440
:100CC000882E7B018C01C601B5012DE133EF41E097
:100CD00050E00E94DC2ECA01B9012CEE34EF4FEF38
:100CE0005FEF0E94882E6E0D7F1D801F911F97FF62
:100CF00004C06150704080409048688379838A8343
:100D00009B839B01AC015F77B901CA01CDB7DEB708
:100D1000EAE00C941B2F0E943B06089581EB92E0C1
:100D20000E943B0608956093B1027093B2028093D3
:100D3000B3029093B4020895A0E0B0E0E2EAF6E0D6
:100D40000C94F82EEC012B016A016115710519F064
:100D5000FB0191838083C114D10449F0C60102973D
:100D6000839728F020E030E040E050E0DCC0A9901C
:100D70008A2D90E00E94482F892BC9F7FDE2AF161B
:100D800021F4A9903324339405C08BE2A81609F40A
:100D9000A9903324C114D10421F0E0E1CE16D1048E
:100DA00011F5F0E3AF1669F48881883711F08835C2
:100DB00041F4A980229682E0382A20E1C22ED12C6B
:100DC00012C0C114D10479F4E0E3AE1659F199E9E7
:100DD000E92E99E9F92E99E9092F99E1192F8AE06D
:100DE000C82ED12C3AC0FAE0CF16D10491F080E1A0
:100DF000C816D10429F0E8E0CE16D104F9F415C0E4
:100E0000BFEFEB2EBFEFFB2EBFEF0B2FBFE01B2F73
:100E100024C0A9E9EA2EA9E9FA2EA9E90A2FA9E135
:100E20001A2F1BC0F8E0CF2ED12CEFEFEE2EEFEFF4
:100E3000FE2EEFEF0E2FEFE11E2F0FC0960144277D
:100E400037FD4095542F6FEF7FEF8FEF9FEF0E949C
:100E5000BA2EC901DA017C018D0120E030E040E0CA
:100E600050E060E03601882477FC8094982C70ED87
:100E7000B72EBA0CF9E0FB1570F48A2D81548A3133
:100E800018F499ECB92E06C08A2D81568A3148F59E
:100E900089EAB82EBA0C8B2D90E08C159D050CF5C7
:100EA0006F3FE9F0E216F30604071507B8F0CA0130
:100EB000B901A40193010E94882E9B01AC018B2DE6
:100EC00090E0A0E0B0E0280F391F4A1F5B1F2817F1
:100ED00039074A075B0710F061E001C06FEFA99086
:100EE000C6CF4114510451F0662311F0219703C07D
:100EF00031FE04C02297F201D183C08330FE07C0C7
:100F000050954095309521953F4F4F4F5F4F67FF6C
:100F10000AC082E290E090934806809347062FEF44
:100F20003FEF4FEF5FEFB901CA01CDB7DEB7E1E1A7
:100F30000C94142FFC0188279927E89421912032E2
:100F4000E9F3293010F02E30C8F32B3241F02D3266
:100F500039F4689404C00E94EF07820F911D21911B
:100F600020532A30C0F31EF4909581959F4F089529
:100F700046E953E00E94BD070895009731F4DA0175
:100F80008D919C91009709F40EC0DC01FB013D910D
:100F90002191222319F03217C9F3FACF332331F408
:100FA000DA011D921C928827992708951197AF9313
:100FB000BF93FB013D912191321771F4332321F44A
:100FC00088279927119702C01E921196FA01A193C2
:100FD000B0839F918F910895222369F7EACF7AE039
:100FE000979F902D879F802D910D112408958091BA
:100FF0009803813019F482E08093980380919803DC
:10100000833019F484E0809398030895009721F1C8
:101010009C0140E050E068E478EE81E090E00E94BE
:10102000DC2EC901DA018F3F9105A105B10531F030
:1010300028F08FEF90E0A0E0B0E008C00097A10595
:10104000B10521F481E090E0A0E0B0E08093B3002E
:101050008091B000806103C08091B0008F7E80934A
:10106000B0000895E3E0F0E089E0809357008491B8
:1010700090E08670863009F491E0892F08951F93DF
:10108000182F0E943208882379F09FB781E080935F
:101090008F05F894A89588E1809360001093600014
:1010A000112309F0A8959FBF1F910895382F20E0C4
:1010B00080912105909122058227932740E061E2EB
:1010C00070E19C01220F331F97FF04C0C9018627DE
:1010D000972701C0C9014F5F483099F790932205C7
:1010E00080932105089586E38093BE0380E092EC0F
:1010F000A1E0B0E08093BF039093C003A093C1032D
:10110000B093C20387E08093CB0380EC92E9ADEE0D
:10111000B9E18093C3039093C403A093C503B09334
:10112000C60385E08093CC038DEE9EEFADEABEED65
:101130008093C7039093C803A093C903B093CA03D5
:10114000ADECB3E080E090E0863010F0E0E004C069
:10115000FC01E058FC4FE081ED9301968831910548
:1011600099F782E08093E5038AE08093E60308958F
:1011700080EC91EDA8E9BBE180939B0390939C03E5
:10118000A0939D03B0939E0310929F031092A0031F
:101190001092A1031092A20308958436910520F4C1
:1011A000BC0180E090E025C08E3B910550F48A554B
:1011B0009040BC0180E090E02AE030E040E050E068
:1011C00016C0823D910550F4845B9040BC0180E0E4
:1011D00090E024E630E040E050E009C08D5C9040B3
:1011E000BC0180E090E028E532E040E050E00E9461
:1011F000882E24E630E040E050E00E94882E0895DA
:1012000090E08C599F4F0E94CD080895DC0198967C
:10121000EC91F0E0E770F070E858FC4F80810895A1
:101220008F929F92AF92BF92CF92DF92EF92FF92F6
:101230000F931F938C010E940609D80197962C9159
:1012400030E043E150E0249FF001259FF00D349FF2
:10125000F00D1124EB54FD4F80809180A280B3806B
:1012600090E00F96AA2797FDA095BA2FBC01CD015B
:1012700020E43FE14DE750E00E94882EA501940153
:101280000E94BA2E69017A0180ED97E0A0E0B0E0FB
:10129000C80ED91EEA1EFB1ED80198968C91887143
:1012A00081F060E07EEE8AEB9BE0A50194010E9454
:1012B000BA2E28513C4F4F4F5F4FC20ED31EE41E33
:1012C000F51E87EE93E0A0E0B0E0C80ED91EEA1E3E
:1012D000FB1EC701B60128EE33E040E050E00E945B
:1012E000BA2ECA01B90128EE33E040E050E00E9476
:1012F000882E1F910F91FF90EF90DF90CF90BF90BD
:10130000AF909F908F9008958F3F910509F010F452
:1013100080E0089522E08030920710F481E0089583
:101320008050934010F083E0089582E00895CF92BA
:10133000DF92FF920F931F93CF93DF93F82FEB0170
:101340006A01182F1695E0E088819981D6018C9367
:101350008A819B8111968C9311978C819D81129625
:101360008C9312978E819F8113968C93139728816B
:1013700039814A815B816C817D818E819F819295CB
:10138000990F990F907C832F8370982B852F8370F2
:10139000880F880F982B872F83708295807F982BDA
:1013A00014969C9385E090E0C80ED91E2896EF5FB6
:1013B0001E1750F6F0FF21C0888199810E94840990
:1013C000F82E8A819B810E948409182F8C819D812F
:1013D0000E948409082F8E819F810E948409F294C3
:1013E000FF0CFF0C70ECF7221295107F1F29182BB1
:1013F000000F000F012BD6010C93DF91CF911F91AD
:101400000F91FF90DF90CF90089523E080329207F4
:1014100018F420E030E026C023E0883E920748F42C
:101420009C012F51334054E0369527955A95E1F7AA
:1014300019C027E0803D920720F49C012C5D3340C9
:1014400011C028E08839920718F02FEF33E00AC066
:101450009C01285C374044E0369527954A95E1F792
:101460002D503C4FC90108959C013695279525754F
:101470003575821B930B9C013695279536952795DC
:101480002373337383739373280F391FC901E4E007
:1014900096958795EA95E1F7820F931F8F709F705D
:1014A00021E031E0AC01429FC001439F900D529F6B
:1014B000900D1124892F0895882339F02D9800006C
:1014C0002B9A00002D9A000008952D9800002B986B
:1014D00000002D9A000008952D9A000083B12D98E8
:1014E000000090E0B4E096958795BA95E1F7817099
:1014F00008950F931F93082F5C9A2D985C9810E025
:10150000802F80780E945C0A000F1F5F1830C1F79F
:101510002D981F910F9108958F770E94790A089551
:101520000F931F93082F10E0802F80780E945C0A91
:10153000000F1F5F1830C1F72D981F910F9108956C
:101540000F931F932D9880E000E0182F110F0E9439
:101550006C0A810F0F5F0830C1F71F910F9108953A
:101560000E948C0A0E94A00A5C9A08951F93162F6D
:1015700080680E94790A812F0E94900A5C9A1F91CC
:1015800008951F931091C7031827EEEBF3E0E80FBF
:10159000F11D89E767850E94B60A8DE3612F0E94DD
:1015A000B60A82E4612F0E94B60A1F91089586E26E
:1015B0000E94B00A08950F931F938C018CE1F801EB
:1015C00064810E94B60A8DE1F80165810E94B60A25
:1015D0008EE1F80166810E94B60A80E2F801678117
:1015E0000E94B60A81E2F80160850E94B60A82E292
:1015F000F80161850E94B60A83E2F80162850E94C3
:10160000B60A84E2F80163850E94B60A85E2F80111
:1016100064850E94B60A8AE2F80165850E94B60ACE
:101620008EE6F80166850E94B60A8FE6F8016785A6
:101630000E94B60A80E7F80160890E94B60A81E735
:10164000F80161890E94B60A82E7F80162890E9466
:10165000B60A1F910F910895EF92FF920F931F9377
:10166000CF93DF937B018C01603028E372072CE974
:1016700082072CE1920728F520E836E948E950E096
:101680000E94BA2EE9016897B90180E090E020E855
:1016900039E647E65FEF0E94882E6E0D7F1D801FA2
:1016A000911F32E0660F771F881F991F3A95D1F777
:1016B00021E732E040E050E00E94BA2E890180E448
:1016C00021C020E03DE241E351E00E94BA2EE90151
:1016D0006897B90180E090E020E033ED4EEC5EEFDA
:1016E0000E94882E6E0D7F1D801F911F660F771F31
:1016F000881F991F21E732E040E050E00E94BA2E97
:10170000890180E69E012F71622F680F85E70E9494
:10171000B60A86E7612F0E94B60A87E7602F0E940B
:10172000B60ACDB7DEB7E6E00C941F2F9F92AF92BA
:10173000BF92CF92DF920F93DF93CF9300D000D070
:10174000CDB7DEB7982E83E00E94B00A8093E703FE
:1017500084E00E94B00A8093E80386E060E00E9483
:10176000B60A87E061E00E94B60A89E06FE70E944E
:10177000B60A8AE065E00E94B60A8BE065E10E9445
:10178000B60A8CE062E10E94B60A8DE06DEF0E941D
:10179000B60A8EE060E00E94B60A992019F084E152
:1017A00093E008C08091E50323E1829FC0011124EA
:1017B0008B549D4F0E94DB0A80E36CE80E94B60ABE
:1017C00082E36FE00E94B60A83E362E40E94B60AF5
:1017D00084E36AE00E94B60A85E36AE20E94B60AE0
:1017E00086E36DE20E94B60A87E364ED0E94B60AC2
:1017F00088E360E00E94B60A89E360E00E94B60ACE
:10180000992049F065E7A62E61ECB62E61ECC62E54
:101810006EEDD62E08C0A090C703B090C803C0904C
:10182000C903D090CA030AE38D2D9927AA27BB27A5
:1018300089839A83AB83BC83802F69810E94B60A17
:10184000802F8B5F69810E94B60ADC2CCB2CBA2CCE
:10185000AA240F5F0E3341F783E46FEF0E94B60AAC
:1018600084E46FEF0E94B60A85E46FEF0E94B60A27
:1018700086E46FEF0E94B60A992019F08DE666E0C3
:1018800003C08DE66091CB030E94B60A89E760E051
:101890000E94B60A8AE76091CC030E94B60A83E7E9
:1018A00060E00E94B60A84E760E00E94B60A9920D0
:1018B00029F060EC72E98DEE99E108C06091C303F4
:1018C0007091C4038091C5039091C6030E942C0BB4
:1018D0000F900F900F900F90CF91DF910F91DF90AD
:1018E000CF90BF90AF909F90089587E061E00E94F5
:1018F000B60A8EE764E20E94B60A88E063E00E94BE
:10190000B60A88E060E00E94B60A87E065E00E94BF
:10191000B60A85E062E00E94B60A83E00E94B00A3F
:101920008093E70384E00E94B00A8093E80308955F
:10193000582F40918C04842F90E0FC01EF70F070E0
:101940009F012F5F3F4F74E0959587957A95E1F75A
:101950002817390751F0E458FB4F5083842F8F5FCD
:101960008F70407F842B80938C0408951F920F9278
:101970000FB60F9211241F932F933F934F935F93B2
:101980006F937F938F939F93AF93BF93CF93DF9387
:10199000EF93FF93C0918600D09187002091CE04F1
:1019A0003091CF048091AD04882309F047C0CE0167
:1019B000821B930B9C0180919F0387FD02C036958B
:1019C000279599E0253C390708F180914703863037
:1019D000D0F0809147038F3FB1F020E00EC0E22F9E
:1019E000F0E0EE0FFF1FDF01A255BB4F8D919C91E0
:1019F000E95DFC4F918380832F5F80914703281717
:101A000070F31092AC041092470318C082E02D3B93
:101A1000380760F180914703803140F5109147030A
:101A2000C9010E94050AE12FF0E0EE0FFF1FE25509
:101A3000FB4F918380831F5F10934703D093CF04A4
:101A4000C093CE04FF91EF91DF91CF91BF91AF9101
:101A50009F918F917F916F915F914F913F912F91C6
:101A60001F910F900FBE0F901F9018958FEF8093CE
:101A70004703E4CF83E0809380008AE9809381006C
:101A800080919F0386FD05C08091810080648093D2
:101A900081008FEF9FEF9093890080938800809161
:101AA0006F00806280936F0008956F3020F08695FC
:101AB0008695805408958DE0689F802D11240895A7
:101AC000882319F460E071E002C063E071E085E210
:101AD00096E00E943C2C0895A0E0B0E0E2E7FDE033
:101AE0000C94012F182F0E940F299B01AC018091AB
:101AF0001B0590911C05A0911D05B0911E05690163
:101B00007A01C81AD90AEA0AFB0AD701C60189581C
:101B10009341A040B04010F010921A0520931B058D
:101B200030931C0540931D0550931E052091AD0474
:101B3000822F81508230E8F580911A05882309F4BC
:101B40004FC1813011F482E0BCC1803108F035C151
:101B5000E82FF0E0E255FB4F10838F5F80931A056A
:101B6000803109F0B0C1A0EBB4E0213039F4119616
:101B7000EC911197E695E6958C9109C08D919C9119
:101B80001197E92FE695E695E69596958795E031CC
:101B900040F4F0E090E0EE0FFF1FE95DFC4F918311
:101BA00080831092AC04129684E0AE3BB807E9F64D
:101BB0008AC1233009F004C180911A05882321F4D9
:101BC0001F3009F080C10CC1883130F4E82FF0E0FB
:101BD000E355FB4F108374C1883109F0EEC0112327
:101BE00009F0EBC0C0E0D0E00BE010E0DE0163E004
:101BF000AA0FBB1F6A95E1F7C09FB001C19F700D8E
:101C0000D09F700D1124FB01E255FB4F8081218193
:101C1000922F977095958795FD01EE0FFF1FE95D57
:101C2000FC4F91838083FB01E155FB4F308136955A
:101C3000369536952181422F4295440F407E842F60
:101C4000832B269526952695922F977095958795A7
:101C5000FD01EE0FFF1FE75DFC4F91838083FB01C9
:101C6000E055FB4F808182958695869583704181F2
:101C7000942F990F990F292F282B42954695469519
:101C8000437082818170880F880F382F342B3595EF
:101C90002795FD01EE0FFF1FE55DFC4F318320838B
:101CA000FB01EE54FB4F308136952181422F479541
:101CB00044274795842F832B2695922F97709595CF
:101CC0008795FD01EE0FFF1FE35DFC4F918380833D
:101CD000FB01ED54FB4F308132953F702181422F43
:101CE0004295407F842F832B22952F70922F9770DF
:101CF00095958795FD01EE0FFF1FE15DFC4F9183E8
:101D00008083FB01EC54FB4F8081881F8827881F4C
:101D10004181942F990F292F282B441F4427441FBA
:101D200082818370880F382F342B35952795FD01DC
:101D3000EE0FFF1FEF5CFC4F31832083FB01EA5461
:101D4000FB4F3081369536952181422F4295440FC5
:101D5000440F407C842F832B26952695922F9770D5
:101D600095958795AA0FBB1FFD01ED5CFC4F9183F4
:101D7000808369547B4FFB01208122952695277033
:101D80004181342F330F330F330F832F822B942F46
:101D900092959695977095958795AB5CBC4F1196EB
:101DA0009C938E932196C230D10509F01FCF80916C
:101DB000C40483FD02C01092AC0410921A0583C0C3
:101DC000243009F080C040911A05442359F4183A90
:101DD000B1F4109222051092210588EA0E9456085B
:101DE00081E06FC0413019F410931F0504C04230E8
:101DF00031F410932005812F0E9456085DC0609138
:101E00002005262F30E0220F331FE42FF0E0C90118
:101E100002968E179F0734F0433268F7E555FB4F63
:101E20001083E9CF2D5F3F4F40912105509122054E
:101E3000E217F30749F4912F80E048275927509380
:101E400022054093210538C0812F90E0481759079B
:101E500089F580911F05813069F5613118F080E1C5
:101E600080932005D09020054EEAE42E44E0F42E25
:101E700000E010E01BC0F701D081C0E0818190E05C
:101E80008C2B9D2B33E0969587953A95E1F70E9430
:101E9000050AF801EE0FFF1FE95DFC4F9183808377
:101EA0000F5F1F4F82E090E0E80EF91E0D1518F34A
:101EB0001092AC0410921A0580911A05882319F02B
:101EC0008F5F80931A05CDB7DEB7E8E00C941D2F25
:101ED000FF920F931F93CF93DF93182F092FF62EA6
:101EE0008EE30E94B60A212F302FC901EC0110E0C9
:101EF00005C08FE769910E94B60A1F5F1F15C8F3DE
:101F000085E064E00E94B60A83E00E94B00A8093F4
:101F1000E70384E00E94B00A8093E8030E940F293F
:101F20006093E9037093EA038093EB039093EC03CF
:101F300087E069E00E94B60A81E080939803CDB7FC
:101F4000DEB7E5E00C94202F0E94680F8091980383
:101F50008130D9F40E940F292091E9033091EA03DE
:101F60004091EB035091EC03621B730B840B950BB8
:101F7000605A76488140904040F4E8CF85E296E090
:101F800067E071E00E943C2C0895809198038130B5
:101F9000A9F3089585E296E06EE70E94F42D089576
:101FA000A0E0B0E0E6EDFFE00C94002F6C0185E2CC
:101FB00096E06EE70E94F42D760100E010E0C0E0AC
:101FC000D0E0B0E2BB2E0AC00830110521F49E011A
:101FD0002095F60120870894E11CF11CF70160812F
:101FE000862F8D57823040F485E296E06DE70E949F
:101FF000F42DF70160816B2585E296E00E94F42DB7
:102000000115110551F0F70180819E01280F311D46
:10201000C32FDD27C20FD31FD0700F5F1F4F0930B2
:10202000110591F6CDB7DEB7E9E00C941C2FA9E0BD
:10203000B0E0EDE1F0E10C94072F382FE62F80910E
:10204000910490E0019664E270E00E94A72E982F20
:102050008093910488E9898380E18A83913071F0CB
:10206000913028F0923099F09330E1F416C085E079
:102070008B8381EF8C832F5F2D8317C09B8381EF30
:102080008C8384E6489FC00111249D830EC084E0A8
:102090008B8381EF8C833D8308C09B8381EF8C838E
:1020A000ED8303C00E94CA0F04C0CE0101960E94B6
:1020B000D00F2996E2E00C94232F0F931F93CF9318
:1020C000DF93182F092F85E296E06EE70E94F42D2A
:1020D000212F302FC901EC0110E000E288818D57DB
:1020E000823040F485E296E06DE70E94F42D88810D
:1020F0008027888385E296E069910E94F42D1F5F16
:10210000193061F785E296E06EE70E94F42DDF91C9
:10211000CF911F910F910895A9E0B0E0E2E9F0E1BD
:102120000C94072F382F80919104882379F48EEF37
:1021300089833A836B83842F90E0959587958C8370
:102140002D83198618861F821E822FC040918C0411
:10215000842F90E09C012F70307054E09595879506
:102160005A95E1F78217930721F18DEF89831A823F
:102170001B82DE01149620E008C0E458FB4F8081EA
:102180008D93405F2F5F263069F0842F90E0FC0133
:1021900034E0F595E7953A95E1F78F709070E81780
:1021A000F90759F740938C042A83CE0101960E94C7
:1021B0005D108091910490E0019666E070E00E94CD
:1021C000A72E809391042996E2E00C94232F9F92EE
:1021D000AF92BF92CF92DF92EF92FF920F931F9335
:1021E000B82EA62ED42EC22E902E0E940F297B012F
:1021F0008C0180917B0420918D0430918E0440915C
:102200008F04509190048823B1F0D801C701821B3C
:10221000930BA40BB50B815E9E42A040B04020F111
:102220002C2DDC1408F42D2D8B2D6A2D422F292DF9
:102230000E94171011C0D801C701821B930BA40B79
:10224000B50B81539547A040B04070F08B2D6A2D9F
:102250004D2D2C2D0E948C10E0928D04F0928E0456
:1022600000938F04109390041F910F91FF90EF90B3
:10227000DF90CF90BF90AF909F90089585E296E059
:102280006091EE030E94F42D08951F93182F85E2AC
:1022900096E0612F0E94F42D8091EE0381278093B8
:1022A000EE031F9108951F93192F0E944511812F4E
:1022B0000E9445111F910895DF92EF92FF920F93B4
:1022C0001F93D82E7B011092EE0305E216E0C801A1
:1022D00065EB0E94F42DC80162E60E94F42D8D2D5D
:1022E0000E944511C7010E9453111F910F91FF9049
:1022F000EF90DF900895A0E0B0E0E1E8F1E10C9408
:10230000FF2E8CE00E94B00A882379F585E296E0E2
:1023100063E171E00E943C2C5E9A80E00E94960B83
:102320000E94750C5E9821C085E296E00E94BB2D4C
:10233000482F8091AD04882321F0842F0E946C0DDA
:1023400014C080911805E82FF0E031969F012F719D
:10235000307031978091170590E02817390729F0E0
:10236000E251FB4F40832093180585E296E00E94DE
:10237000812D892BC9F680919803843009F08CC097
:102380000E940F2960939C0470939D0480939E0487
:1023900090939F04611571058105910561F481E0B9
:1023A00090E0A0E0B0E080939C0490939D04A09303
:1023B0009E04B0939F048091A8049091A904816029
:1023C0009093A9048093A80483E0809398038FE7F7
:1023D0000E948C0AC5EED4E00E94A00A899304E012
:1023E000CE3ED007C9F74091D0048091E504282F54
:1023F00030E0842F90E08227932786FF40C080E45E
:1024000048274093D004C90188739070C89709F594
:1024100010E014C01F5F8091E603E12FF0E084FF1D
:1024200006C0EB51FB4F80810E94980C07C0EB5116
:10243000FB4F85E296E060810E94F42D212F30E071
:102440008091E50490E0877090708217930714F7ED
:1024500016C02F733070232B91F48091E604809383
:10246000A0048091E7048093A2048091E804809303
:10247000A3048091EB048093AA041092AB04809192
:102480001905813019F482E08093190580911905AE
:10249000833011F4109219050E940F295B016C0121
:1024A0008091A4049091A504A091A604B091A704E2
:1024B0000097A105B105C9F0A6019501281B390BAC
:1024C0004A0B5B0BDA01C901885B9B40A040B0401E
:1024D00060F00E94D70A8093A1041092A404109285
:1024E000A5041092A6041092A7048EEB93E00E941C
:1024F0001009209198043091990440919A045091C8
:102500009B0486017501E21AF30A040B150BE6160B
:10251000F7060807190708F4EAC0A0929804B092D9
:102520009904C0929A04D0929B04A8958091AC041F
:10253000883008F0D4C08091AC048F5F8093AC04E5
:10254000E0909C04F0909D0400919E0410919F04E3
:10255000E114F1040105110511F18EEB93E00E94E5
:102560001009AE18BF08C00AD10A6A157B058C0590
:102570009D0588F480919F0385FD04C080ED97E060
:102580000E94060810929C0410929D0410929E04D2
:1025900010929F0404C080E090E00E940608909191
:1025A000D004907C9093D0040091180510911705E9
:1025B0000117B1F180911905823091F590589093EF
:1025C000D0048EEB93E00E940609893010F048E0B9
:1025D00002C0482F415030E013C03F5FA32FB0E04E
:1025E000812F90E0FC01E251FB4F2081FD01E0537F
:1025F000FB4F2083A25FBA4F2C930196182F1F71B7
:10260000341710F4101749F710931705832F895CBE
:102610009091D004892B8093D00430930E051AC07A
:10262000209119052430D1F490910E05EFE0F5E0EA
:10263000A1EDB4E0292F30E02E0F3F1F02C08191A1
:102640008D93E217F307D9F7995C8091D004982B0A
:102650009093D00483E08093190523C08091930464
:10266000823029F491609093D0045E9A0FC09093C9
:10267000D0045E98222319F481E08093190580919B
:102680001905833019F484E080931905F89480913A
:10269000E603877067E273E041ED54E00E9497091A
:1026A00078945D9A809192040E94C10A8EEB93E027
:1026B0000E940609682F80ED94E00E94680FE09167
:1026C0009204EF5FE0939204E83131F0F0E0E254DD
:1026D000FC4F8785882359F41092920408C080919A
:1026E000AC04883009F45E9A89E08093AC04809150
:1026F000E603887171F180919803823051F58091E1
:10270000A8049091A904880F991F9093A90480931D
:10271000A80483E0809398030E94750C0E940F29FF
:102720006093A4047093A5048093A6049093A704D7
:10273000611571058105910561F481E090E0A0E0EB
:10274000B0E08093A4049093A504A093A604B09352
:10275000A7048091E60384FF1EC08091A804909195
:10276000A9048E7F0E94340A182F8091A0046091E2
:10277000AA040E94550D082F8091A104612F0E9488
:10278000550D282F8091A2046091A304402F009141
:1027900099030E94E7105D98809193048130C9F0FD
:1027A000813020F0823009F03FC033C08EE00E94BB
:1027B000332A892BC9F581E0809393040E94012973
:1027C0006093940470939504809396049093970477
:1027D0002BC08EE00E94332A892B21F50E9401290B
:1027E000209194043091950440919604509197045F
:1027F000621B730B840B950B695E734080409040A5
:1028000098F082E08093930480ED97E00E940608A0
:102810000BC08EE00E94332A892B31F080E090E0DB
:102820000E94060810929304CDB7DEB7EAE00C943C
:102830001B2F8CE060E00E9494298BE061E00E94F5
:1028400094298DE061E00E94942982E060E00E947A
:10285000942984E061E00E949429089582E08093A5
:10286000B00085E08093B10083E061E00E9494298C
:1028700083E060E00E94002A08951F93182F0E94B1
:102880000F2960938D0470938E0480938F0490932E
:10289000900410937B04112329F440E855E260E092
:1028A00070E004C040E051EE60E070E085E296E048
:1028B0000E94FA2C1F910895ACE1B0E0E2E6F4E149
:1028C0000C94FF2E0E940F297B018C0181E00E9455
:1028D000960BA4E7AA2E6E010894C11CD11CF3E04C
:1028E000BF2EA982C60161E00E94A40FB092980396
:1028F0000E94750C6AEF70E080E090E00E9435293C
:1029000080919803833009F07DC085E296E00E94B3
:10291000812D892B09F076C00E940F296E197F093D
:10292000800B910B6058734C894C914008F06AC041
:10293000D8CF8FE70E948C0A0E94A00A843509F044
:102940005CC089830E94A00A182F00E010937A04CB
:10295000009379040E94A00A080F111D10937A04B5
:10296000009379040E94A00A809378040E94A00A30
:1029700080937704813108F040C0FF2407C00E9493
:10298000A00A095A1B4FF8018083F3940F2D10E021
:102990008091770490E0880F991F0817190778F342
:1029A00080E78983CE01019661E00E94A40F83E055
:1029B000809398030E94750C62E370E080E090E0E1
:1029C0000E943529809198038330A9F08FE70E94F7
:1029D0008C0A0E94A00A803581F4898303EA13E0FF
:1029E0000E94A00AF80181938F01F3E00E3B1F07BC
:1029F000B9F781E003C082E001C083E06C96EAE0B1
:102A00000C941B2F80919803833009F092CFF3CF61
:102A100083E00E94B00A8093E70384E00E94B00A3A
:102A20008093E80387E061E00E94B60A6AE070E004
:102A300080E090E00E9435290E94750C0000089506
:102A40000F931F93082F17C05E9A64E670E080E032
:102A500090E00E9435295E9864E670E080E090E0A6
:102A60000E9435291F5F101778F36CE271E080E057
:102A700090E00E94352910E0F6CF482F392F25E04D
:102A80000DC0F999FECF1FBA842F932F92BD81BD3F
:102A900060BD0FB6F894FA9AF99A0FBE215059F01A
:102AA000F999FECF842F932F92BD81BDF89A80B5FE
:102AB000681739F7089582E00E9420150895A0E074
:102AC000B0E0E5E6F5E10C94F82E482E562EEE2403
:102AD000FF2488249924C0E0D0E0CC24DD2436E310
:102AE000332E04C055245394CC24DD24442069F4AF
:102AF00080919903839DE00111242AE9E22E23E0CD
:102B0000F22E99E0892E912C1DC021E0421671F41D
:102B100080919903839DE00111242B968EEBE82E82
:102B200083E0F82E09E2802E912C0CC032E043168F
:102B300049F419E9E12E13E0F12EB1E08B2E912C2E
:102B4000C8EDD0E03E016C0C7D1C10922205109265
:102B50002105E3011BC0552059F4F999FECFD2BDE0
:102B6000C1BDF89A80B5F701E00FF11F808307C05F
:102B7000F701E00FF11FCE0160810E943D150E0D9F
:102B80001F1DF80180810E94560821969E0126197A
:102B9000022F10E008151905F0F2CE015520D9F4E6
:102BA000F999FECFD2BDC1BDF89A20B5F999FECFF3
:102BB0002196D2BDC1BD2197F89A80B590E0B22E82
:102BC000AA248A299B2920912105309122052817C2
:102BD000390759F487CF2196609122050E943D154F
:102BE000CE01609121050E943D1580E091E0C80E64
:102BF000D91E91E0C91693E0D90608F477CF852D48
:102C0000CDB7DEB7E1E10C94142F80E061E00E94C3
:102C10005F1581E061E00E945F15089580E060E04B
:102C20000E945F15882331F081E060E00E945F150B
:102C3000882331F40E94B8080E9473080E94051688
:102C4000089582E061E00E945F15089582E060E0EF
:102C50000E945F1580919903843020F010929903AF
:102C60000E94211608951F93182F0E942616809106
:102C70009903811731F0143020F4109399030E94C6
:102C800021161F9108951092550485E6E0EFF3E0B8
:102C9000DF011D928A95E9F708951F93182F8F374A
:102CA00011F08830E1F5E0915504EE2309F455C0A8
:102CB000E150E0935504F0E0E051FC4F108285E2D2
:102CC00096E06DE00E94F42D10E00AC0E12FF0E0E4
:102CD000E051FC4F85E296E060810E94F42D1F5F79
:102CE00080915504181790F385E296E060E20E9407
:102CF000F42D85E296E06DE00E94F42D10E00AC00C
:102D0000E12FF0E0E051FC4F85E296E060810E9407
:102D1000F42D1F5F80915504181790F31CC08B3160
:102D200019F40E9443161FC08D30E9F08A30D9F0A3
:102D300080915504843688F485E296E0612F0E94E4
:102D4000F42D80915504E82FF0E0E051FC4F108302
:102D50008F5F8093550480E007C085E296E067E0CE
:102D60000E94A82AF8CF81E01F9108951F93CF9366
:102D7000DF93CDECD3E010E03BC085E296E062E269
:102D800071E00E94392C85E296E0612F4AE050E024
:102D90000E94B62B85E296E06FE271E00E94392C2A
:102DA000699170E080E090E02091CC0330E040E059
:102DB00050E00E94882E20E137E240E050E00E947F
:102DC000882EDC01CB014091C3035091C403609174
:102DD000C5037091C603480F591F6A1F7B1F85E208
:102DE00096E02AE030E00E947D2B1F5F183119F039
:102DF0008881882311F6DF91CF911F910895EF927A
:102E0000FF920F931F93882339F485E296E066E6DC
:102E10007AE00E94C62A3BC090E00E94CD0824E6DA
:102E200030E040E050E00E94BA2E122F032FF42E23
:102E3000E52E622F732F842F952F2AE030E040E09B
:102E400050E00E94BA2E85E296E0BA01A9012AE07C
:102E500030E00E946E2B85E296E06EE20E94A82A86
:102E6000612F702F8F2D9E2D2AE030E040E050E042
:102E70000E94BA2EAB01BC0185E296E02AE030E068
:102E80000E946E2B85E296E063E70E94DA2A1F918A
:102E90000F91FF90EF900895FF920F931F93CF93A0
:102EA000DF9385E296E06CE57AE00E94872A8091C4
:102EB000A303813041F485E296E063E47AE00E9466
:102EC000C62AFF2466C0823029F485E296E06CE2CF
:102ED0007AE0F5CF8430A9F785E296E068E17AE000
:102EE000EECFCF2DD0E0C930D1051CF06F2D685C3E
:102EF00002C06F2D6F5C85E296E00E94A82A85E2F1
:102F000096E060E17AE00E94872ABE016F5F7F4F02
:102F100085E296E04AE050E00E94122C85E296E0BD
:102F200065E07AE00E94872A8E010D551C4FD8017A
:102F30001196EC91E032F8F485E296E068EF79E0E2
:102F40000E94872AF8018181803130F085E296E085
:102F500063E371E00E94392CCD55DC4F698170E04C
:102F60006F7070706F5F7F4F85E296E04AE050E0CF
:102F70000E94252C0DC0F0E0EF70F070EE0FFF1FE7
:102F8000E85BFC4F6081718185E296E00E943C2CF9
:102F9000F39480917804F81608F4A3CF85E296E0C4
:102FA0006DED79E00E94872A8091BB030E94FF1695
:102FB00085E296E062EC79E00E94872A8091BC036A
:102FC0000E94FF1685E296E067EA79E00E94872A70
:102FD0008091BD030E94FF1685E296E06CE879E0DF
:102FE0000E94872A4091B3035091B4036091B503C6
:102FF0007091B603411551056105710539F185E2FE
:1030000096E02AE030E00E947D2B85E296E069E5BB
:1030100079E00E94872A8091B7030E940009AB01E2
:10302000BC0185E296E02AE030E00E947D2B85E23B
:1030300096E065E379E00E94872A85E296E0609158
:10304000B8034AE050E00E94C82B06C085E296E033
:103050006CE279E00E94C62A85E296E06FE079E0B2
:103060000E94872A6091B9037091BA0385E296E0C5
:103070004AE050E00E94A22B85E296E062EF78E001
:103080000E94872A6091B203603150F470E06F5F54
:103090007F4F85E296E04AE050E00E94252C06C072
:1030A00085E296E069EE78E00E94C62A85E296E025
:1030B0006CEC78E00E94872A8091B10380FD03C008
:1030C00065E371E002C069E371E085E296E00E9489
:1030D0003C2C85E296E06FEA78E00E94872A809196
:1030E000B10382700E94600D85E296E060E978E0AD
:1030F0000E94872A8091B10384700E94600D85E24E
:1031000096E061E778E00E94872A8091B103887099
:103110000E94600DCDB7DEB7E5E00C94202F1F9321
:10312000CF93DF9385E296E060EB7BE00E94872AF5
:103130004091C3035091C4036091C5037091C603CD
:1031400085E296E02AE030E00E947D2B85E296E061
:103150006AE97BE00E94872A4091C7035091C80327
:103160006091C9037091CA0385E296E020E130E0E6
:103170000E947D2B85E296E064E87BE00E94872A2E
:1031800085E296E06091CB034AE050E00E94C82BB4
:1031900085E296E06EE67BE00E94872A85E296E073
:1031A0006091CC034AE050E00E94C82B85E296E093
:1031B00068E57BE00E94872ACDECD3E010E012C0E6
:1031C000112331F085E296E06DE371E00E94392C25
:1031D00085E296E069914AE050E00E94B62B1F5FBD
:1031E000183119F08881882359F785E296E00E940A
:1031F000B02A85E296E062E47BE00E94872A85E2BD
:1032000096E06091E5034AE050E00E94C82B85E219
:1032100096E06DE27BE00E94872AE091E603F0E011
:10322000E770F070EE0FFF1FE859FC4F608171816D
:1032300085E296E00E943C2C85E296E068E17BE026
:103240000E94872A8091E60390E088719070883010
:10325000910589F0893091051CF4892B39F01BC048
:103260008031910569F04897B1F40FC085E296E08E
:103270006FE07BE00EC085E296E063E07BE009C092
:1032800085E296E06DEF7AE004C085E296E063EFB8
:103290007AE00E94C62A85E296E06FED7AE00E940D
:1032A000872A4091BF035091C0036091C103709180
:1032B000C20385E296E02AE030E00E947D2B85E2A1
:1032C00096E066EC7AE00E94872A80919F038072E4
:1032D0000E94600D85E296E06DEA7AE00E94872AFE
:1032E00080919F0380740E94600D85E296E064E9FE
:1032F0007AE00E94872A80919F0380780E94600D67
:1033000085E296E067E77AE00E94872A8EEB93E0F9
:103310000E941009AB01BC0185E296E02AE030E092
:103320000E946E2B85E296E062E77AE00E94872A8F
:103330008EEB93E00E9410099B01AC0160E472E403
:103340008FE090E00E94BA2E85E296E0BA01A901D2
:103350002AE030E00E946E2B85E296E06FE67AE08C
:103360000E94C62ADF91CF911F910895EF92FF929C
:103370000F931F938C0175E2E72E76E0F72EC701BD
:10338000612F70E04AE050E00E94912BC7016EE28D
:103390000E94A82A64E0169507956A95E1F70F70D8
:1033A0001070C701B8014AE050E00E94912B1F91B4
:1033B0000F91FF90EF9008950F931F93CF93DF939A
:1033C0002091EF032F3FA9F585E296E061EF75E0CC
:1033D0000E94872A80E693E00E94B61985E296E073
:1033E00060ED75E00E94872A8091790490917A04BB
:1033F0000E94B61985E296E06DE975E00E94C62A42
:1034000085E296E06AE775E00E94C62A85E296E0CA
:1034100062E675E00E94C62A85E296E06DE375E0FB
:103420000E94C62A85E296E00E94B02A0E944C17AC
:1034300069C012160CF066C0332727FD30958091C5
:10344000780490E0821793070CF45CC085E296E064
:1034500068E275E00E94872A6091EF03772767FD95
:10346000709585E296E04AE050E00E94252C85E2C6
:1034700096E06DEF74E00E94872A08E210E03AC0FF
:10348000C12FD0E0CC0FDD1FC95ADB4F288130E0BF
:103490008091EF03992787FD9095019728173907A9
:1034A00041F585E296E06FE371E00E94392C85E2F8
:1034B00096E0602F4AE050E00E94B62B85E296E04D
:1034C00063E471E00E94392CE981F0E0EF70F07064
:1034D000EE0FFF1FE85BFC4F6081718185E296E093
:1034E0000E94392C85E296E067E471E00E94392C55
:1034F0000F5F1F5F80917704181710F285E296E046
:103500000E94B02ADF91CF911F910F910895ACE1F5
:10351000B0E0EDE8FAE10C94012F282F8091EF0341
:103520008F3F09F042C1822F90E0FC013A97EF36BD
:10353000F10508F033C1EC5CFF4F0C942E2F85E2AF
:1035400096E069E471E0AEC085E296E069E471E07E
:103550000E943C2C1CC185E296E065E571E00E946A
:103560003C2C85E78983DE011296E3EAF3E08BE1E8
:1035700001900D928150E1F7CE0101966CE10E941D
:10358000A40F0E94750C83E08093980368EC70E0B0
:1035900080E090E00E94352980919803843009F002
:1035A000FDC08FE70E948C0A0E94A00A898385359E
:1035B00009F0F4C085E296E06FED74E00E94C62A3F
:1035C00085E296E061EC74E00E94C62A85E296E00E
:1035D00063EA74E0ACC085E296E06DE671E00E94BB
:1035E0003C2C89E68983CE01019661E00E94A40FFC
:1035F0000E94750C83E08093980368EC70E080E093
:1036000090E00E94352980919803843009F0C6C06B
:103610008FE70E948C0A0E94A00A89838E010E5FA8
:103620001F4F9DE1E92EF12CEC0EFD1E0E94A00A19
:10363000D8018D938D01AE15BF05C1F7A3EAB3E0A4
:10364000FE0132968BE101900D928150E1F7898164
:10365000893409F0A3C085E296E065E874E00E9431
:10366000C62A85E296E067E674E00E94C62A85E2F3
:1036700096E069E474E05BC085E296E067E871E09B
:103680000E943C2C8EEF8093EF0388C0205227507D
:10369000922F905380917804891738F485E296E050
:1036A00066E971E00E943C2C79C09093EF036FC0F3
:1036B00084E18093EF0385E296E062E174E037C035
:1036C00085E18093EF0385E296E06BED73E02FC018
:1036D00086E18093EF0385E296E064EA73E027C019
:1036E00087E18093EF0385E296E06AE573E01FC00F
:1036F00088E18093EF0385E296E069E473E017C008
:1037000089E18093EF0385E296E065E373E00FC003
:103710008AE18093EF0385E296E060E273E007C000
:103720008BE18093EF0385E296E068EF72E00E9400
:10373000C62A34C085E296E06EED72E00E94C62A89
:103740008091B10391E01DC085E296E068EC72E0E3
:103750000E94C62A8091B10392E013C085E296E0F0
:1037600063EB72E00E94C62A8091B10394E009C025
:1037700085E296E068E972E00E94C62A8091B10372
:1037800098E089278093B1038FEF8093EF030E9425
:10379000DC1904C085E296E00E94BB2D85E296E02C
:1037A0000E94812D892BB1F763C1822F0E944D1693
:1037B000882309F45DC180915504882321F48FEF9B
:1037C0008093EF034DC180EF93E060E070E040E054
:1037D00050E00E949C069B01AC016091EF03862F94
:1037E000992787FD9095A92FB92FFC013197EB31CF
:1037F000F10508F025C1ED55FF4F0C942E2FE62F53
:10380000FF27E7FDF0958091780490E08E179F07E1
:103810000CF416C1DA01C9010197A109B109809719
:10382000A105B10540F0FF2410E008E26F01089403
:10383000C108D10826C0ED55FC4F822F81508083EE
:10384000E7C0612F70E0660F771F695A7B4FFB015D
:10385000808190E08C159D0599F4802F90E0A0E088
:10386000B0E082179307A407B50749F4F601ED55B8
:10387000FC4FDB0111968C918183FF24F3940F5F41
:103880001F5F809177041817E0F2C0C02F3F310509
:103890004105510511F008F0D3C02093BB03B8C017
:1038A0002F3F31054105510511F008F0C9C02093A3
:1038B000BC03AEC02F3F31054105510511F008F0A2
:1038C000BFC02093BD03A4C08091F0038062803705
:1038D00019F581EF93E060E070E040E050E00E9475
:1038E0009C069B01AC01DC01CB010197A109B10948
:1038F0000897A105B10508F0B6C0CA01B90124EDC9
:1039000030E340E050E00E94882E9B01AC012A5E2B
:103910003C4A4A46554E24C0863611F581EF93E065
:1039200060E070E040E050E00E949C069B01AC012A
:10393000DC01CB010197A109B1090797A105B105E8
:1039400008F091C0CA01B90128EA31E640E050E030
:103950000E94882E9B01AC01245E3C434E46544E8F
:10396000211531054105510561F0DA01C901805485
:10397000914EAD49B8418158904FAA4FB24008F0DE
:103980005FC02093B3033093B4034093B5035093C7
:10399000B6033EC02F3F31054105510511F008F037
:1039A0004FC02093B70334C0DA01C9010197A109C0
:1039B000B1098F3F9105A105B10508F041C02093E1
:1039C000B80326C0DA01C901845C9940A040B04028
:1039D0008D549D41A040B04038F43093BA032093F9
:1039E000B903FF24F39401C0FF24211531054105DB
:1039F000510511F48FEF07C0213131054105510503
:103A000028F4822F81508093B20302C0FF20C1F0BE
:103A1000809156048823D1F48091C7039091C80304
:103A2000A091C903B091CA030196A11DB11D809355
:103A3000C7039093C803A093C903B093CA0306C0F9
:103A400085E296E068EA71E00E943C2C0E944316F1
:103A50008FEF8093EF0385E296E06AE00E94DA2A16
:103A60000E94DC1905C021E030E040E050E07DCF4D
:103A70006C96E8E00C941D2F85E296E06CE472E011
:103A80000E94C62A85E296E064E372E00E94C62A9C
:103A900085E296E00E94812D892B31F085E296E047
:103AA0000E94BB2D0E94871A0E945C14823019F07C
:103AB000833069F405C085E296E066E172E004C0F7
:103AC00085E296E06FEF71E00E94C62A08958FEFBD
:103AD0008093EF03109256040E94DC190CC085E21B
:103AE00096E00E94812D892B31F085E296E00E94BC
:103AF000BB2D0E94871A8091EF038E3F81F70895B6
:103B00008091EF03992787FD9095A92FB92FFC018C
:103B10003196EB30F10508F074C0E254FF4F0C947D
:103B20002E2F85E296E064E678E00E94C62A80E6C1
:103B300093E00E94B61985E296E06CE478E00E947A
:103B4000C62A85E296E067E278E00E94C62A85E20E
:103B500096E06DEF77E00E94C62A85E296E06CED74
:103B600077E00E94C62A85E296E06FEA77E00E943D
:103B7000C62A85E296E069E877E00E94C62A85E2D7
:103B800096E065E677E00E94C62A85E296E06EE35D
:103B900077E00E94C62A85E296E00E94B02A0E9441
:103BA0008F182FC085E296E061E277E028C085E2B9
:103BB00096E06CEF76E023C085E296E067EE76E073
:103BC0001EC085E296E068EC76E019C085E296E0DA
:103BD00064E876E014C085E296E06FE676E00FC018
:103BE00085E296E06AE576E00E94C62A85E296E0E4
:103BF00064E176E004C085E296E06EEF75E00E9435
:103C0000C62A6AE070E080E090E00E94352904C096
:103C100085E296E00E94BB2D85E296E00E94812D10
:103C2000892BB1F70895A2E2B0E0E9E1FEE10C943E
:103C3000F72E8E010F5F1F4F80E1D8011D928A95EC
:103C4000E9F785E296E066EC71E00E943C2C0E9468
:103C5000081520E431EE4DE958E12F8F38A349A330
:103C60005AA380EC91EDA8E9BBE18B8F9C8FAD8FBF
:103C7000BE8F24EF31E040E050E02F8B388F498F2A
:103C80005A8F50E5C52E53ECD52EE12CF12C40E493
:103C9000442E41EE542E4DE9642E48E1742E8824C2
:103CA0009924540133241E8A1D8A198A1A8A1B8A70
:103CB0001C8AFFC085E296E00E94BB2D8434B9F0D7
:103CC000853430F48332B9F18C3209F0CCC044C071
:103CD000833509F0C8C02F8D38A149A15AA1C90167
:103CE000DA012C013D01882499245401E2C085E2C7
:103CF00096E064E40E94A82A85E296E040E451EE52
:103D00006DE978E12AE030E00E94DC2B85E296E064
:103D10006CE20E94A82A85E296E040EC51ED68E949
:103D20007BE12AE030E00E94DC2B85E296E06CE249
:103D30000E94DA2ABEC019821A821B821C821D824E
:103D40001E821F82188619861A861B861C861D866F
:103D50001E861F86188A3AC0339434E0331609F061
:103D6000A8C069817A818B819C8128EE33E040E094
:103D700050E00E94882E6F8F78A389A39AA36D814B
:103D80007E818F8198850E94882E6B8F7C8F8D8F8E
:103D90009E8F89859A85AB85BC858F8B988FA98FDF
:103DA000BA8F6D857E858F8598890E94882E6B01DC
:103DB0007C0190E2C9169EE4D90690E0E90690E005
:103DC000F90630F48CE162E30E94B60A332471C034
:103DD000A0E3CA16A5E7DA06A0E0EA06A0E0FA0624
:103DE00018F48CE162E2F0CFB0E4CB16BCE9DB065C
:103DF000B0E0EB06B0E0FB0618F48CE166E2E4CF3D
:103E0000E0E5CE16E3ECDE06E0E0EE06E0E0FE06DE
:103E100018F48CE162E1D8CFF0E6CF16FAEEDF06B7
:103E2000F0E0EF06F0E0FF0618F48CE165E1CCCF9E
:103E300020E7C21621E1D20621E0E20620E0F206E8
:103E400018F48CE161E0C0CF30EAC31636E8D3063F
:103E500031E0E30630E0F30618F48CE163E0B4CF20
:103E60008CE165E0B1CF30ED232E280E49E04215FC
:103E700000F1032D10E0000F111F000F111F81E052
:103E800090E08C0F9D1F080F191FD8016D917D9137
:103E90008D919C912AE030E040E050E00E94882E15
:103EA000620D711D811D911DF801608371838283F4
:103EB000938385E296E00E94812D892B09F0FACE4A
:103EC00081149104A104B10489F4C301B2010E94D8
:103ED0002C0B61E070E080E090E00E943529FFEF5C
:103EE000FE8B1D8A198A1A8A1B8A1C8A2F89388D93
:103EF000498D5A8D82169306A406B506E0F40E94F9
:103F0000D70A29893A894B895C89280F311D411DBF
:103F1000511D298B3A8B4B8B5C8B3D89381708F4EC
:103F20008D8B4E89841708F48E8B0894811C911C0C
:103F3000A11CB11C56C0C301B20128EE33E040E021
:103F400050E00E94BA2E85E296E0BA01A9012AE06B
:103F500030E00E946E2B85E296E06CE20E94A82A77
:103F600085E296E06D894AE050E00E94B62B85E23A
:103F700096E06CE20E94A82A69897A898B899C89DB
:103F8000A50194010E94BA2E85E296E0BA01A9012A
:103F90002AE030E00E946E2B85E296E06CE20E94FF
:103FA000A82A85E296E06E894AE050E00E94B62B8E
:103FB00085E296E06CE20E94DA2A4C0C5D1C6E1CD5
:103FC0007F1C8B8D9C8DAD8DBE8D84159505A605B2
:103FD000B70520F44F8C58A069A07AA088249924B2
:103FE00054012F8D38A149A15AA1285E3340404089
:103FF000504009F05ECFA296E2E10C94132FAAE59F
:10400000B0E0E5E0F0E20C94032F8B017A018A30F6
:1040100009F4EDC08B3010F5853009F47EC0863090
:1040200080F4823009F453C0833020F4813009F0E9
:1040300029C23CC0833009F45BC0843009F022C23D
:104040005FC0873009F48FC0873008F482C08830A1
:1040500009F491C0893009F015C295C0893609F478
:1040600061C18A3680F4863609F40CC1873620F4A3
:10407000853609F007C2EDC0873609F41CC18836C1
:1040800009F000C220C18C3609F4A3C18D3638F482
:104090008A3609F452C18B3609F0F4C18EC18D36CF
:1040A00009F4CBC1873C09F0EDC1DFC181E069E2D1
:1040B00070E00E945C110EEB13E0F80181918F011A
:1040C0000E944511F3E0073E1F07B9F7E3C182E004
:1040D0006BE170E00E945C1103EA13E0F80181914A
:1040E0008F010E944511F3E00E3B1F07B9F7D2C1C3
:1040F00083E061E070E00E945C110E945C14C8C122
:1041000084E061E070E00E945C1181E00E94451152
:104110000E943E110E94131EBFC16091770470E09F
:10412000660F771F85E00E945C1100E010E008C078
:10413000F801E95AFB4F80810E9445110F5F1F4F24
:104140008091770490E0880F991F0817190780F372
:10415000A1C186E062E070E00E945C1180E693E01D
:104160000E94531197C187E061E070E00E945C11EA
:10417000809178048DC188E061E070E00E945C115C
:104180008091990385C186E68983CE01019661E01D
:104190000E94A40F0E94750C83E08093980368EC42
:1041A00070E080E090E00E9435298091980384308F
:1041B000E1F48FE70E948C0A0E94A00A898386346A
:1041C00071F489E060E270E00E945C1110E00E94EE
:1041D000A00A0E9445111F5F1032C9F75BC189E038
:1041E00061E070E00E945C11A6C089E04CC18AE0E9
:1041F00069E070E00E945C1110929A0380918F0533
:10420000882351F080919F039091A003A091A10376
:10421000B091A203806809C080919F039091A00390
:10422000A091A103B091A2038F7780939F039093F5
:10423000A003A093A103B093A2030AE913E0F8013D
:1042400081918F010E944511F3E0033A1F07B9F7EE
:1042500021C185E661E070E00E945C110932110520
:1042600009F015C120E030E0F901E254FC4FD7011C
:10427000A20FB31F8C9180832F5F3F4F29323105EE
:1042800099F759C086E661E070E00E945C110B313D
:10429000110509F0FCC020E030E0F901ED55FC4FBC
:1042A000D701A20FB31F8C9180832F5F3F4F2B311B
:1042B000310599F740C087E661E070E00E945C112B
:1042C0000E94051638C088E661E070E00E945C112B
:1042D00085E78A83DE011396E3EAF3E08BE1019040
:1042E0000D928150E1F7CE0102966CE10E94A40F7D
:1042F0000E94750C83E08093980360E273E080E095
:1043000090E00E94352980919803843009F0BFC065
:104310008FE70E948C0A0E94A00A8A83853509F0E3
:10432000B6C009C089E661E070E00E945C110E949D
:1043300073080E94B80881E0ABC08AE661E070E0D3
:104340000E945C1189E68E8FCE014E9661E00E943C
:10435000A40F0E94750C83E08093980360E273E0E1
:1043600080E090E00E94352980919803843009F024
:104370008EC08FE70E948C0A0E94A00A8E8F8E0149
:10438000015E1F4F6AE3E62EF12CEC0EFD1E0E942B
:10439000A00AF80181938F01EE15FF05C1F7A3EA8A
:1043A000B3E0FE017F968BE101900D928150E1F721
:1043B0008E8D893409F06BC0BECF8BE661E070E072
:1043C0000E945C11F70180810E9433160E940E1634
:1043D000B2CF8CE661E070E00E945C110032110502
:1043E00071F487E68AAFDE01DB96F70180E2019087
:1043F0000D928150E1F7CE01CA9661E205C087E4D3
:104400008AAFCE01CA9661E00E94A40F0E94750C8B
:1044100083E0809398036CE474E080E090E00E9475
:10442000352980919803843091F58FE70E948C0A9A
:104430000E94A00A873459F57ECF8DE661E070E0D6
:104440000E945C110930110511F520E030E0F901FE
:10445000E656FC4FD701A20FB31F8C9180832F5FCC
:104460003F4F2930310599F766CF87EC61E070E066
:104470000E945C1181E00E9445110E943E11109241
:10448000ED030AC08AEC61E070E00E945C1180E0FC
:104490000E9445110E943E11C65ADF4FE6E00C947F
:1044A0001F2FA0E0B0E0E7E5F2E20C94FF2E84E0DD
:1044B000A82E06E0B02E15E0C12E03E215E0B4E60A
:1044C000DB2EA2E0EA2EF3E0FF2EA1C085E296E00B
:1044D0000E94BB2D982F80938E0580918D0583308F
:1044E00021F1843028F4813099F08230B8F409C089
:1044F000853009F448C0853020F1863009F087C046
:104500005FC0953B09F083C081E080938D057FC03B
:10451000923609F07AC0E0928D0579C090938C05AF
:1045200090938B05F0928D0572C09093890510923F
:104530008A0580918B05892780938B05A0928D0534
:1045400066C0D92FC0E02091890530918A052C2BB7
:104550003D2B30938A052093890580918B0589270F
:1045600080938B05C0928D052536310508F44FC028
:104570008CEC61E070E00E945C1181E00E944511CA
:104580000E943E1142C02091870530918805F901B3
:10459000ED5DFA4F908380918B05892780938B0581
:1045A0002F5F3F4F309388052093870580918905C1
:1045B00090918A052817390750F1B0928D0527C0D0
:1045C00080918B05891759F4609187057091880552
:1045D00080918C0543E255E00E94FF1F0DC08BECDB
:1045E00062E070E00E945C1180918C050E94451190
:1045F0008091EE030E944511F8018D2D11928A954C
:10460000E9F7109288051092870510928D0585E2D2
:1046100096E00E94812D892B09F058CFCDB7DEB7E7
:10462000EAE00C941B2F81E08093ED0308C085E243
:1046300096E00E94812D892B11F00E9451228091D9
:10464000ED038823A1F70895A0E0B0E0EAE2F3E2E9
:104650000C94022F0E940F296115710581059105A7
:10466000C9F30E9493061092C7031092C8031092D8
:10467000C9031092CA03DD24E090C703F090C80379
:104680000091C9031091CA03102F0F2DFE2CEE24A8
:104690000E948E062FEF30E040E050E00E94DC2EBA
:1046A000E60EF71E081F191FE092C703F092C80319
:1046B0000093C9031093CA03D39444E0D416E1F6DF
:1046C000CDECD3E000E010E090E1E92E97E2F92E86
:1046D0004EC00F5F19F40E9473084DC00E948E06F1
:1046E00022E330E040E050E00E94DC2E6F5FEDEC12
:1046F000F3E090E004C08191861759F39F5F911712
:10470000D0F38091CC0390E08E9D90018F9D300D71
:104710009E9D300D1124862F90E0AC01249FC00196
:10472000259F900D349F900D1124AA2797FDA095E9
:10473000BA2F2091C3033091C4034091C503509117
:10474000C603820F931FA41FB51F20919B033091B6
:104750009C0340919D0350919E03281739074A07F7
:104760005B0708F4B6CF69931F5F183121F0888189
:10477000882309F0AECFCDB7DEB7E7E00C941E2F4B
:104780001F931091EF031F3F09F0F1C0893409F422
:1047900067C08A3428F5883309F479C0893368F40E
:1047A000803309F486C0813308F06FC08B3109F47F
:1047B0004DC0813209F0D5C03DC0813409F49AC0A2
:1047C000823438F4893309F472C0803409F0C9C0E6
:1047D00031C0823409F4A1C0863409F0C2C052C08D
:1047E000823609F49AC0833690F4883579F1893598
:1047F00038F4823509F43FC0833509F0B2C01FC0D8
:104800008A3509F4A9C0813609F0ABC073C082377C
:1048100091F1833730F48636A9F1893609F0A1C0C9
:104820001FC0883799F08A3709F496C0833709F09A
:1048300098C005C085E296E069E471E019C00E9465
:10484000051685E296E063ED71E006C00E940E1643
:1048500085E296E06DEE71E00E943C2C8EEF7FC009
:104860000E9473080E94B80885E296E06CE072E04E
:104870000E943C2C76C00E94242385E296E065E2EB
:1048800072E0F6CF0E94B6166CC0805368C085E215
:1048900096E06CEE71E00E94C62A9091E603892FA3
:1048A000885F8871977E892B8093E60320C089E01A
:1048B00056C085E296E069ED71E00E94C62A8091BB
:1048C0009F039091A003A091A103B091A20320E2C5
:1048D00030E040E050E082279327A427B52780935B
:1048E0009F039093A003A093A103B093A2031093FE
:1048F000EF0337C085E296E063EC71E00E94C62AC0
:1049000080919F039091A003A091A103B091A20375
:1049100020E430E040E050E012C085E296E062EB37
:1049200071E00E94C62A80919F039091A003A091FC
:10493000A103B091A20320E830E040E050E08227DC
:104940009327A427B52780939F039093A003A09358
:10495000A103B093A20302C00E943C1D8FEF80937D
:10496000EF038091EF038E3F09F4DDC0D4C00E94B5
:104970004D16882309F4D7C080915504882321F46B
:104980008FEF8093EF03C7C080EF93E060E070E0AB
:1049900040E050E00E949C069B01AC018091EF0337
:1049A000992787FD9095A92FB92FFC013197E93000
:1049B000F10508F08CC0E753FF4F0C942E2FDA015D
:1049C000C9018154914EAD49B8418F57904FAA4FBC
:1049D000B24008F07CC02093C3033093C4034093DB
:1049E000C5035093C6039AC02093C7033093C803EE
:1049F0004093C9035093CA0381E0809356048EC04C
:104A0000283031054105510508F061C02093CB03E2
:104A100085C0DA01C9010197A109B1090A97A10569
:104A2000B10508F054C02093CC0378C080EF93E028
:104A30006DE371E00E94B80710E00EC0183130F449
:104A4000E12FF0E0E254FC4F87871F5F80E090E0A9
:104A50006DE371E00E94B807009759F00E949A0731
:104A6000009761F706C0E12FF0E0E254FC4F178693
:104A70001F5F1831C0F352C0253031054105510583
:104A800030F52093E5034AC0DA01C9010197A10975
:104A9000B1090697A105B105D0F48091E603887F9E
:104AA000822B8093E6033AC0DA01C9010197A1097C
:104AB000B1098050924CA140B04048F42093BF030C
:104AC0003093C0034093C1035093C20327C085E2D3
:104AD00096E068EA71E00E943C2C13C08091C70305
:104AE0009091C803A091C903B091CA030196A11D7A
:104AF000B11D8093C7039093C803A093C903B093DB
:104B0000CA030E9443168FEF8093EF0385E296E07D
:104B10006AE00E94DA2A0E94801D05C08091560436
:104B20008823E1F2EECF1F9108958FEF8093EF037A
:104B3000109256040E94801D0CC085E296E00E94EF
:104B4000812D892B31F085E296E00E94BB2D0E94D9
:104B5000C0238091EF038E3F81F76AE070E080E030
:104B600090E00E94352904C085E296E00E94BB2DAA
:104B700085E296E00E94812D892BB1F70895AAE283
:104B8000B0E0E5ECF5E20C94FC2E0E9401297B01DB
:104B90008C0181E00E94960B04C085E296E00E94A1
:104BA000BB2D85E296E00E94812D892BB1F75E989E
:104BB000DD24D39452E6752E42E0842E912C8C0E87
:104BC0009D1E5E010894A11CB11C33E0C32E0E94FF
:104BD000012920E030E06E197F09800B910B693CC0
:104BE00071058105910510F021E030E08D2D90E0F8
:104BF00028233923232B99F10E9401297B018C0161
:104C00005D9A80ED97E00E9406087982D401EEEB70
:104C1000F3E089E201900D928150E1F7C5016AE26B
:104C20000E94A40F5D9880E090E00E940608C09268
:104C300098030E94750C62E370E080E090E00E94AF
:104C4000352980919803843051F4C09298038FE7FE
:104C50000E948C0A0E94A00A823409F4DD248EE0AE
:104C60000E94332A892B49F5DD24D39426C05E9A0D
:104C70005D9A85E296E00E94BB2D8D30910569F02A
:104C80008E3091051CF40A97B1F407C08332910568
:104C900069F08234910579F40CC085E296E064EA0B
:104CA00071E00E94C62A0E94952505C00E94131E2D
:104CB00002C00E9413235E985D9885E296E00E94F0
:104CC000812D892B09F483CFD2CF8F929F92AF92FF
:104CD000BF92CF92DF92EF92FF920F931F938EE0DD
:104CE0000E94332A892B09F083C068EC70E080E0D1
:104CF00090E00E94352980E090E00E9406080E9422
:104D000001295B016C0160ECE62E62E1F62E012DBB
:104D1000112DEA0CFB1C0C1D1D1D06C08EE00E940F
:104D2000332A892B09F062C00E9401296E157F0584
:104D30008007910798F38EE00E94332A892B09F0AF
:104D400055C080ED97E00E9406080E9401297B0172
:104D50008C0199249394882488E496E2A0E0B0E042
:104D6000A80EB91ECA1EDB1E29C0AE14BF04C006A1
:104D7000D10638F480ED97E00E94060888248394D9
:104D80001DC00E9401296E197F09800B910B693C9F
:104D900071058105910590F00E9401297B018C012C
:104DA00080E0992009F481E0982E882319F480E0AE
:104DB00090E002C080ED97E00E9406088EE00E941D
:104DC000332A892B91F280E090E00E940608882027
:104DD00049F0809199038F5F83700E9433160E947F
:104DE0000E1606C00E9424230E9405160E94BF25AD
:104DF0001F910F91FF90EF90DF90CF90BF90AF90F9
:104E00009F908F90089580E067EF77E042E050E058
:104E10000E943C280895EF92FF920F931F9380E029
:104E20000E943F080E94191489E061E00E949429C1
:104E300089E060E00E94002A86E061E00E949429F7
:104E400085E061E00E9494298EE060E00E94942950
:104E500088E060E00E94942988E061E00E94002AD6
:104E600081E161E00E94942981E160E00E94002AD2
:104E70000E942E1485E296E040E052EC61E070E082
:104E80000E94FA2C0E9426160E940E160E943A0DCD
:104E90008FEF8093AC040E94032778940E9401292D
:104EA0007B018C018091AC048F3F09F0DBC00E9434
:104EB00001296E197F09800B910B605D774080405E
:104EC000904008F0CFC0EECF85E296E00E94BB2D67
:104ED00085E296E00E94812D892BB1F785E296E06C
:104EE00062E472E00E94392C80E693E00E94B619D9
:104EF00085E296E069E572E00E94392C85E296E051
:104F000064E070E04AE050E00E94252C68EC70E01C
:104F100080E090E00E94352985E296E00E94812D94
:104F200004970CF185E296E00E94BB2D8234910536
:104F3000D1F485E296E00E94BB2D8E34910599F460
:104F400085E296E00E94BB2D8434910561F485E2F0
:104F500096E00E94BB2D819731F480E090E00E94A2
:104F600006080E94BF254091BF035091C003609185
:104F7000C1037091C203DB01CA010197A109B10904
:104F80000497A105B10568F44093AD04433029F0BE
:104F900040E052EC61E070E004C040EA56E861E0B5
:104FA00070E085E296E00E94FA2C0E9465265E98E9
:104FB00080E090E00E9406080E943A0D80E00E9486
:104FC000960B809192040E94C10A0E94750C109267
:104FD000170510921805109219056CE271E080E037
:104FE00090E00E94352980ED97E00E94060864E673
:104FF00070E080E090E00E94352980E090E00E941F
:10500000060810E015C064E670E080E090E00E94C1
:10501000352980ED97E00E94060864E670E080E0A4
:1050200090E00E94352980E090E00E9406081F5F12
:1050300080919903181738F38091E60390E084FF7C
:1050400009C020E088719070489709F421E0822F10
:105050000E943D148FE00E943F081F910F91FF9026
:10506000EF90089580ED97E00E9406088EE061E0E1
:105070000E94002A5E9A2CCF823000F5E82FF0E0E3
:10508000EE0FFF1FE057FA4F71836083882319F0FA
:105090008130A1F408C0809169008C7F842B8093BB
:1050A0006900E89A089580916900440F551F440FE4
:1050B000551F837F842B80936900E99A08951F927E
:1050C0000F920FB60F9211242F933F934F935F933C
:1050D0006F937F938F939F93AF93BF93EF93FF93C0
:1050E0008091900590919105892B29F0E091900590
:1050F000F09191050995FF91EF91BF91AF919F912B
:105100008F917F916F915F914F913F912F910F9070
:105110000FBE0F901F9018951F920F920FB60F920F
:1051200011242F933F934F935F936F937F938F93AC
:105130009F93AF93BF93EF93FF93809192059091CC
:105140009305892B29F0E0919205F091930509953B
:10515000FF91EF91BF91AF919F918F917F916F914F
:105160005F914F913F912F910F900FBE0F901F9025
:1051700018951F920F920FB60F9211242F933F9301
:105180008F939F93AF93BF938091980590919905CA
:10519000A0919A05B0919B0530919C050196A11DA7
:1051A000B11D232F2D5F2D3720F02D570196A11D06
:1051B000B11D20939C058093980590939905A09329
:1051C0009A05B0939B058091940590919505A091C7
:1051D0009605B09197050196A11DB11D8093940588
:1051E00090939505A0939605B0939705BF91AF91C5
:1051F0009F918F913F912F910F900FBE0F901F9015
:1052000018958FB7F89420919805309199054091A1
:105210009A0550919B058FBFB901CA0108959FB7A8
:10522000F894209194053091950540919605509100
:10523000970586B5A89B06C08F3F21F02F5F3F4F93
:105240004F4F5F4F9FBF542F432F322F2227280FDE
:10525000311D411D511D82E0220F331F441F551F78
:105260008A95D1F7B901CA010895EF92FF920F9381
:105270001F93CF93DF937B018C010E940F29EB01D9
:105280000EC00E940F296C1B7D0B685E7340C8F333
:105290000894E108F10801091109C851DC4FE11433
:1052A000F1040105110569F7CDB7DEB7E6E00C940E
:1052B0001F2F789484B5826084BD84B5816084BDDD
:1052C00085B5826085BD85B5816085BDEEE6F0E07F
:1052D000808181608083E1E8F0E0108280818260DB
:1052E0008083808181608083E0E8F0E0808181605C
:1052F0008083E1EBF0E0808184608083E0EBF0E08C
:10530000808181608083EAE7F0E08081846080832F
:1053100080818260808380818160808380818068D9
:1053200080831092C1000895CF93DF93482F50E0FF
:10533000CA018850944FFC0134914C51544FFA01EA
:105340008491882369F190E0880F991FFC01EA534A
:10535000F44FA591B491FC01E053F44FC591D49161
:10536000662351F42FB7F8948C91932F909589234D
:105370008C93888189230BC0623061F42FB7F89435
:105380008C91932F909589238C938881832B88838C
:105390002FBF06C09FB7F8948C91832B8C939FBF2F
:1053A000DF91CF910895833071F0843028F48130FB
:1053B000A1F0823021F514C08630B1F08730D1F0F1
:1053C0008430E9F404C0809180008F7703C080911D
:1053D00080008F7D80938000089584B58F7702C010
:1053E00084B58F7D84BD08958091B0008F778093C0
:1053F000B00008958091B0008F7D8093B000089533
:10540000FF920F931F93F62E482F50E0CA01845F3E
:10541000934FFC012491CA018850944FFC011491D0
:105420004C51544FFA0104910023C9F0222319F082
:10543000822F0E94D329E02FF0E0EE0FFF1FE053F0
:10544000F44FA591B4919FB7F894FF2021F48C916B
:105450001095812302C08C91812B8C939FBF1F914B
:105460000F91FF9008950F931F93482F50E0CA01AA
:10547000845F934FFC012491CA018850944FFC0132
:1054800004914C51544FFA011491112319F420E066
:1054900030E015C0222319F0822F0E94D329812FDA
:1054A00090E0880F991F8652944FFC01A591B4910A
:1054B0008C9120E030E0802311F021E030E0C90140
:1054C0001F910F910895A0E0B0E0E9E6FAE20C9494
:1054D000012F7C016B018A01C0E0D0E00FC0D60132
:1054E0006D916D01D701ED91FC910190F081E02D5E
:1054F000C7010995C80FD91F0150104001151105AA
:1055000071F7CE01CDB7DEB7E8E00C941D2FEF9216
:10551000FF920F931F93CF93DF937C018B01C0E029
:10552000D0E0F8010F5F1F4F6491662359F0D70157
:10553000ED91FC910190F081E02DC7010995C80F14
:10554000D91FEFCFCE01CDB7DEB7E6E00C941F2F09
:10555000DC01ED91FC910190F081E02D0995089519
:10556000EF92FF920F931F938C016DE00E94A82A87
:105570007C01C8016AE00E94A82A9C012E0D3F1DF3
:10558000C9011F910F91FF90EF900895EF92FF9244
:105590000F931F937C010E94872A8C01C7010E94F0
:1055A000B02A9C01200F311FC9011F910F91FF905C
:1055B000EF900895EF92FF920F931F937C010E944A
:1055C000A82A8C01C7010E94B02A9C01200F311F1C
:1055D000C9011F910F91FF90EF900895CF93DF9332
:1055E000EC016115710519F420E030E00FC0DB011A
:1055F0000D900020E9F71197A61BB70BE881F98100
:105600000280F381E02DAD0109959C01C901DF9174
:10561000CF9108954F925F927F928F929F92AF9217
:10562000BF92CF92DF92EF92FF920F931F93DF937F
:10563000CF93CDB7DEB7A1970FB6F894DEBF0FBEFC
:10564000CDBF2C01742ECB01223008F42AE019A220
:1056500031E2C32ED12CCC0EDD1E822E9924AA2439
:10566000BB24672D752FA50194010E94BA2E7901E4
:105670008A01C801B701A50194010E94882E472D17
:10568000461B0894C108D1084A3010F4405D01C09F
:10569000495CF6014083E114F1040105110521F094
:1056A0007E2C5F2DC801DDCFC201B6010E94EE2A1B
:1056B000A1960FB6F894DEBF0FBECDBFCF91DF919C
:1056C0001F910F91FF90EF90DF90CF90BF90AF9020
:1056D0009F908F907F905F904F900895DC012115EF
:1056E000310541F4ED91FC910190F081E02D642FA2
:1056F000099508950E940A2B0895EF92FF920F9347
:105700001F937C010E946E2B8C01C7010E94B02A5E
:105710009C01200F311FC9011F910F91FF90EF9045
:105720000895EF92FF920F931F939A017B0100E07F
:1057300010E0B801A7010E946E2B1F910F91FF90FE
:10574000EF900895EF92FF920F931F937C010E94B8
:10575000912B8C01C7010E94B02A9C01200F311FA0
:10576000C9011F910F91FF90EF900895EF92FF9262
:105770000F931F939A01E62EFF2400E010E0B8017A
:10578000A7010E946E2B1F910F91FF90EF9008953B
:10579000EF92FF920F931F937C010E94B62B8C0116
:1057A000C7010E94B02A9C01200F311FC9011F911F
:1057B0000F91FF90EF900895A0E0B0E0E2EEFBE2E1
:1057C0000C94012FEC016A017B012115310541F494
:1057D000E881F9810190F081E02D642F09951BC0CB
:1057E0002A303105B1F477FF13C06DE20E94A82A78
:1057F0008C0144275527BA014C195D096E097F09B0
:10580000CE012AE00E940A2B9C01200F311F04C008
:105810002AE00E940A2B9C01C901CDB7DEB7E8E05F
:105820000C941D2FEF92FF920F931F937B019A010F
:105830000027F7FC0095102FB801A7010E94DC2B70
:105840001F910F91FF90EF900895EF92FF920F93A9
:105850001F937C010E94122C8C01C7010E94B02A68
:105860009C01200F311FC9011F910F91FF90EF90F4
:1058700008950E94EE2A0895EF92FF920F931F93CE
:105880007C010E94392C8C01C7010E94B02A9C0126
:10589000200F311FC9011F910F91FF90EF900895C4
:1058A00008951F920F920FB60F9211242F933F93DA
:1058B0004F938F939F93EF93FF938091C00082FD4E
:1058C0001DC04091C6002091DD053091DE052F5F9F
:1058D0003F4F2F7330708091DF059091E0052817BE
:1058E000390771F0E091DD05F091DE05E356FA4FDE
:1058F00040833093DE052093DD0502C08091C60011
:10590000FF91EF919F918F914F913F912F910F9028
:105910000FBE0F901F9018951F920F920FB60F9207
:1059200011242F933F938F939F93EF93FF93209195
:105930002106309122068091230690912406281793
:10594000390731F48091C1008F7D8093C10014C06C
:10595000E0912306F0912406EF51FA4F20818091C7
:1059600023069091240601968F73907090932406DD
:10597000809323062093C600FF91EF919F918F9112
:105980003F912F910F900FBE0F901F901895A0E0A0
:10599000B0E0EDECFCE20C94FD2EFC0113821282CF
:1059A00088EE93E0A0E0B0E084839583A683B7837C
:1059B0008AE893E091838083758764875787468759
:1059C000318B208B138B028BF58AE48AD78AC68AA7
:1059D000B18EA08E938E828E8F85848F8889858FDD
:1059E0008989868F8A89878F8B8980A32096ECE0AE
:1059F0000C94192FAF92BF92DF92EF92FF920F9308
:105A00001F93CF93DF93EC017A018B01DD244030AB
:105A100081EE580780E0680780E0780711F0DD2408
:105A2000D39491E0A92EB12CEC89FD89DD2069F099
:105A3000C50108A002C0880F991F0A94E2F780836D
:105A400060E079E08DE390E005C0108260E874E8E2
:105A50008EE190E0A80197010E94BA2E21503040BB
:105A600040405040569547953795279580E1203026
:105A7000380720F0DD2011F0DD24D6CFE889F98940
:105A80003083EA89FB89208319A2EE89FF8940814E
:105A900021E030E0C9010C8C02C0880F991F0A94E4
:105AA000E2F7482B4083EE89FF894081C9010D8CC4
:105AB00002C0880F991F0A94E2F7482B4083EE89B1
:105AC000FF894081C9010E8C02C0880F991F0A947A
:105AD000E2F7482B4083EE89FF8980810F8C02C05A
:105AE000220F331F0A94E2F7209528232083DF91A9
:105AF000CF911F910F91FF90EF90DF90BF90AF90EB
:105B00000895DC011C96ED91FC911D97E05CFF4F20
:105B10002191319180819181281B390B2F73307035
:105B2000C901089585E296E00E94812D892B11F02C
:105B30000E94502C0895DC011C96ED91FC911D975C
:105B4000E05CFF4F20813181E054F040DF01AE5B2B
:105B5000BF4F8D919C9111972817390719F42FEF9A
:105B60003FEF07C08D919C91E80FF91F8081282F8E
:105B700030E0C9010895DC011C96ED91FC911D9760
:105B8000E05CFF4F20813181E054F040DF01AE5BEB
:105B9000BF4F8D919C9111972817390719F42FEF5A
:105BA0003FEF10C08D919C911197E80FF91F208154
:105BB0008D919C91119701968F73907011969C9383
:105BC0008E9330E0C9010895DC0191968C919197F4
:105BD000882339F05496ED91FC915597808186FF8A
:105BE000F9CF91961C920895CF93DF93EC01EE8547
:105BF000FF85E05CFF4F20813181E054F0402F5F52
:105C00003F4F2F733070DF01AE5BBF4F8D919C9182
:105C1000119728173907D1F3E05CFF4F80819181FC
:105C2000E054F040E80FF91F6083EE85FF85E05CEB
:105C3000FF4F31832083EE89FF89208181E090E04E
:105C40000F8C02C0880F991F0A94E2F7282B20833B
:105C500081E089A3EC89FD8980818064808381E073
:105C600090E0DF91CF9108958F929F92AF92BF9273
:105C7000CF92DF92EF92FF920F931F9300D000D04C
:105C80000F92EDB7FEB7319684E0ADB7BEB711966F
:105C90008C9383E0818387E0828385E0838381E046
:105CA000848385E296E06DE975E041EE55E025ECF0
:105CB00030E004EC10E0B0ECEB2EF12CA1ECCA2E9D
:105CC000D12CF2ECAF2EB12CE6EC8E2E912C0E9452
:105CD000C72C0F900F900F900F900F901F910F9166
:105CE000FF90EF90DF90CF90BF90AF909F908F90FC
:105CF0000895CF93DF930E9459290E940B27C2E990
:105D0000DDE20E947B112097E1F30E94922DF9CFF2
:105D1000629FD001739FF001829FE00DF11D649F8F
:105D2000E00DF11D929FF00D839FF00D749FF00D1B
:105D3000659FF00D9927729FB00DE11DF91F639FBC
:105D4000B00DE11DF91FBD01CF011124089597FB8E
:105D5000092E07260AD077FD04D086D006D0002071
:105D60001AF4709561957F4F0895F6F79095819597
:105D70009F4F0895A1E21A2EAA1BBB1BFD010DC067
:105D8000AA1FBB1FEE1FFF1FA217B307E407F507EB
:105D900020F0A21BB30BE40BF50B661F771F881FC7
:105DA000991F1A9469F760957095809590959B015D
:105DB000AC01BD01CF01089597FB092E05260ED039
:105DC00057FD04D0D7DF0AD0001C38F45095409519
:105DD000309521953F4F4F4F5F4F0895F6F79095BF
:105DE0008095709561957F4F8F4F9F4F08952F92AB
:105DF0003F924F925F926F927F928F929F92AF925B
:105E0000BF92CF92DF92EF92FF920F931F93CF93A7
:105E1000DF93CDB7DEB7CA1BDB0B0FB6F894DEBF3E
:105E20000FBECDBF09942A88398848885F846E8464
:105E30007D848C849B84AA84B984C884DF80EE80AE
:105E4000FD800C811B81AA81B981CE0FD11D0FB6B7
:105E5000F894DEBF0FBECDBFED010895EE0FFF1F1A
:105E60000590F491E02D0994AA1BBB1B51E107C0DA
:105E7000AA1FBB1FA617B70710F0A61BB70B881FDA
:105E8000991F5A95A9F780959095BC01CD01089569
:105E9000911106C0803219F089508550D0F70895CD
:0A5EA000992788270895F894FFCF92
:105EAA004E6F005965730054582074696D656F759B
:105EBA007421006D6F64756C65206C6F636B65642B
:105ECA003F00486F70206368616E6E656C20002029
:105EDA0040200053004E2F4100386368002C002CEC
:105EEA00205B005D20280029004E4F5420454E417A
:105EFA00424C45440053656E64696E67207365744D
:105F0A0074696E677320746F2052580A0052657361
:105F1A00657474696E672073657474696E6773203B
:105F2A006F6E2052580A0041626F72746564206570
:105F3A00646974730A00696E76616C6964207365BA
:105F4A006C656374696F6E000D0A496E76616C69DF
:105F5A006420696E707574202D20646973636172A0
:105F6A006465642107007363616E6E6572206D6FEC
:105F7A0064650053657474696E677320736176652E
:105F8A006420746F20454550524F4D0A0052657681
:105F9A0065727465642073657474696E67732066CC
:105FAA00726F6D20454550524F4D0A004C6F616427
:105FBA00656420666163746F7279206465666175D1
:105FCA006C74730A004B657920616E6420636861A2
:105FDA006E6E656C732072616E646F6D697A65644A
:105FEA000A004F70656E4C52536E672054582073E6
:105FFA0074617274696E672000206F6E20485720A2
:10600A000050504D005253534900534441005343EA
:10601A004C00525844005458440041494E004C42E6
:10602A004545500053504B54524D0053425553006E
:10603A0053554D44004C4C494E440000342B340017
:10604A003800382B340031320031322B34003136EB
:10605A000001000000C01200001A400AA1204EA54B
:10606A00001B1E27522C23308025000005400AA160
:10607A00204EA50020244EA52C2330004B000006FC
:10608A00400AD0009D49007B289D492C233000E11D
:10609A00000005400A4501D7DC03B81E0EBF0023E5
:1060AA002E48E801008A400A6001555502AD1E20BB
:1060BA00000023C88025000005400AA1204EA50043
:1060CA0020244EA52C233000020002000200020008
:1060DA0002000200020002000200020002000200A6
:1060EA0002000200020002FF610265026A026E02F9
:1060FA00720276027A027E0284028B029002950272
:10610A009B029B029B029B0235019C02A002A202F7
:10611A00A602A902AE02350100070B0C10111500E8
:10612A00160A1322312900000000F42D632A812D5A
:06613A00BB2D9B2DE42D9E
:00000001FF
